:020000040800F2
:10500000A01A0020D5500008D1860008B17D000804
:105010000000000000000000000000000000000090
:10502000000000000000000000000000A190000847
:105030000000000000000000C58E00089D910008DF
:10504000E7500008E7500008E7500008E750000864
:10505000E7500008155B0008E7500008E75000081B
:1050600000000000E7500008515A0008E75000080F
:10507000E7500008C182000800000000E750000867
:1050800000000000E75000080000000000000000E1
:10509000E750000800000000E7500008E750000853
:1050A000E7500008E7500008E7500008859A00081C
:1050B000E7500008E7500008000000000000000072
:1050C0000348854600F060FC0048004755A80008EA
:1050D000A01A00200448804704480047FEE7FEE786
:1050E000FEE7FEE7FEE7FEE739920008C150000840
:1050F00030B50B46014600202022012409E00D4670
:10510000D5409D4205D31D469540491B25469540F7
:1051100040191546521E002DF1DC30BDF0B51FB40C
:105120000646002082B005464024019100901BE015
:10513000019922460F46304600F04EFB049A059B2B
:10514000801A994110D310461946224600F034FBCC
:10515000361A8F410197224601200021009F00F05E
:105160002BFB38184D4100902046641E0028DFDCE0
:10517000019B00982946324607B0F0BD03460B4319
:105180009B0703D009E008C9121F08C0042AFAD2FD
:1051900003E00B780370401C491C521EF9D2704783
:1051A000D2B201E00270401C491EFBD270470022BF
:1051B000F6E710B513460A4604461946FFF7F0FF16
:1051C000204610BD30B504460020034600E05B1CBD
:1051D000934203D2E05CCD5C401BF8D030BDF8B503
:1051E00002464A40D40F42004B0052085B089A42E4
:1051F00002D20246084611464A0023D0C30D4A0097
:10520000DDB2120EAD1A202D35DA49020126490A07
:10521000F6058A19002C00D0524220214F1B11465E
:10522000B9402A411018C20D9A4221D0002C17D043
:10523000012D08DCDA05801AD20F8019D207DBB203
:1052400000F0F6FAF8BDDA05801A012340001B06CB
:10525000C01880185A428018CA0F1043490007E04E
:105260004908C2071143DA05801A801940088018DE
:1052700000F0D6FAF8BD61000122511A001BF7E7D1
:105280000122D2075140AAE70122D2075040A6E7E7
:1052900070B502464A40D50F40004A00ED0740086D
:1052A0005208002814D0002A12D0C40DD30D410298
:1052B0000120C0055202490A520AE41A09181218BC
:1052C0007D34914201D3641C00E04900002C01DAD6
:1052D000002070BD0023914201D3891A0343400886
:1052E00049000028F7D100290AD0914202D10121BA
:1052F000C90705E0914201D2012101E00121C94322
:10530000E005C018401900F08BFA70BDF0B50746F3
:105310000846584087B0C00F049048000E46590018
:1053200040084908BC1A884105D2384631461E4615
:1053300017460B4602465800400810434CD0300D2B
:10534000039040055900400D490D0590401A029008
:10535000402872DA18030121000B09050843019067
:1053600004980092002805D00199524200208841FB
:1053700000920190029840210A1A0199009800F0C9
:105380001BFA05460C466B4607CB00F036FAC019EF
:105390007141039A0E0D0023D71756401A467A40E2
:1053A000164344D0049A002A2DD0029A012A039A67
:1053B00015DC1205C01A914101263605001C714109
:1053C000D20F059ED2070093019202962A462346E9
:1053D00000F074FA07B0F0BD38463146FAE716051A
:1053E000224A0F46B218C01AB74101210905001C14
:1053F0004F4100187F41114618187941E20F1043C0
:105400006D19644113E0E2076D0815436408C20793
:105410001443039A01261205C01A91413605001C57
:105420007141CE07400830434908C01851412A460F
:10543000234600F036FACDE7FFE70498012240004A
:10544000C117121A00238B4104983146C417381A29
:10545000A141EEE730B40124E407634030BC55E7D6
:1054600030B40124E407614030BC4FE70000E0FFA6
:10547000F0B51FB488B00B990998002448400999E9
:10548000C00F490049080991C0070B9900904900D5
:1054900049080B9109990898A64608431CD00B9916
:1054A0000A98084318D0099801244000420D48008A
:1054B000410D099824050003000B204309900B9827
:1054C0000003000B20430B9050181C494018002289
:1054D00001901446104605E0002001460DB0F0BDD5
:1054E000032801DA034600E003239C46C11A0AAEF2
:1054F0000AE05F0008ADED5B4F00F75B7D430027DE
:10550000AA187C41491C5B1E6145F2DD410004ABD9
:105510005A522104120C0A43240C401C0828DFDBD9
:10552000019802900099704601910090059B049AA1
:105530000799069800F0C2F9D0E700000DFCFFFFC4
:10554000F0B50C465C4085B0E40FE40703944C00D2
:1055500000266408590094464908024602962243F0
:1055600021D062460A431ED06200570D4A000E0346
:105570002303550D012402462C492405781B1B0BDF
:10558000360B401823432643614600901C46501AB0
:10559000B44103D30098401C009002E09218009898
:1055A0005B41002803DA0020014605B0F0BD002071
:1055B000012109050746864611E064461D46141B75
:1055C000B54106D36546521BB341744607430C43AD
:1055D000A646CD0740084908284392185B41054676
:1055E0000D43EAD11046184313D060461946504087
:1055F0007140084306D06046101AB34106D201221A
:10560000002306E000220123DB0702E00122D2434F
:105610005310009874460105381C6141029C039D9B
:105620000019694100F03DF9BFE70000FD030000EB
:10563000C217C10F504010B54018CA079623002169
:1056400000F0F6F810BD10B500229623114600F0C8
:10565000EFF810BD0EB5C217C10F5040CA07401871
:105660000021054B0293019200910A460B4600F07F
:1056700025F903B000BD0000330400000EB5054954
:105680000291002100910A460B46019100F016F9A3
:1056900003B000BD33040000410040020122400A73
:1056A000D205090E80187F2901DA0020704796295B
:1056B00003DC9622511AC8407047963988407047DB
:1056C00070B5CD0F4A0009030123090B1B051943CF
:1056D0000B4BED070024520D9A4201DA002070BDF9
:1056E000074B34339A4203DC9A1A00F075F802E053
:1056F0000449511888402C43F1D0404270BD00004D
:10570000FF030000CDFBFFFF4A0009030123090B43
:105710001B051943094B10B5520D9A4201DA0020BE
:1057200010BD064B34339A4203DC9A1A00F054F849
:1057300010BD03495118884010BD0000FF03000050
:10574000CDFBFFFFC20FD207400040080BD0C10DB8
:105750000723DB01C91840020905400A1143C208AA
:10576000400711437047002001467047CB0FDB070D
:10577000490010B5490802460A4307D00A0D07241C
:105780000903E401090B121B002A01DC002010BDF3
:10579000C900440F0C43C100E018D205801800F086
:1057A0003FF810BD0122D207002800DB101A0029A3
:1057B00000DB511A8142704710B5202A04DB0146F4
:1057C000203A9140002010BD914020239C1A0346AE
:1057D000E3401943904010BD10B5202A04DB084671
:1057E000203AD040002110BD0B46D340D0402024A9
:1057F000A21A91400843194610BD10B5202A06DBB5
:10580000CB170846203A1041C1170B4306E00B4660
:105810001341D0402024A21A91400843194610BDDC
:10582000002904DA401C490001D1400840007047BB
:1058300070B40024050C05D11024000402D1002905
:1058400021D01124050E01D100020834050F01D129
:105850000001241D850F01D18000A41C002801DB5C
:105860004000641C002908D020252E1B0D46F54061
:10587000A14000D001212943084301061B1B000A57
:10588000DB1D02D5002070BC7047DB05181880189E
:105890000029F8DA401C4900F5D170BC40084000EE
:1058A000704710B5002B08DA0024401C61419218A3
:1058B0005B411A4301D14008400010BDF0B51FB450
:1058C00082B005460C0003D0084604F099F902E0C6
:1058D00004F096F920300246009021462846FFF752
:1058E0006BFF049B059A04460F4618431143084377
:1058F00014D0184610431BD0009840210A1A1846AD
:105900000599FFF769FF05460E46009A0599049828
:10591000FFF752FF084305D0012004E02046394636
:1059200007B0F0BD0020C11705430E432C43374399
:1059300000990E986305401A7905E40A00220C4389
:10594000FD0A0A3002D500200146E9E701051019D9
:1059500069410C9C0D9D00196941FFF7A2FFDFE72B
:1059600010B5002904DB0124E40740428C412146A4
:10597000002B04DB1C460123DB075242A341994262
:1059800000D1904210BD0000064C0125064E05E0F6
:10599000E36807CC2B430C3C98471034B442F7D350
:1059A000FFF792FBE0AB000800AC000838B50446F6
:1059B000064805490068FFF79BFB604300E0401E76
:1059C00000900028FBD138BD40420F00F8000020B5
:1059D000F8B50446006881688907890F012902D15A
:1059E0000168C90722D18168114A1026114001259A
:1059F00000290ED18168294381600120FFF7D6FF7D
:105A000000F0AAFF07460CE000F0A6FFC01B0A2822
:105A100007D9606D30436065A06D2843A065012003
:105A2000F8BD20680068C043C007EDD10020F8BD74
:105A30001700008010B500231A4603E0845CE318C9
:105A40009BB2521C8A42F9D3D84380B210BD0000E9
:105A500010B5034800F036FD024800F033FD10BDDC
:105A60003C160020F415002030B5446C1C252C4059
:105A70000125A540046C6560046863608368102B91
:105A8000036803D099600068C26030BD9A60006806
:105A9000C16030BD10490120487202205E31487259
:105AA00003203C39487204200E3948720A4B0B49D6
:105AB0005A1C0878587149789971233318715971B3
:105AC000203318775977107551751A461E321075A4
:105AD00051751076517670472C110020E00000209F
:105AE00010B503F0B3FA202003F04EFB012004F0C0
:105AF00037FC002003F048FB044804F0D5FA0448C2
:105B000004F07EFD002004F0B3FD10BDA8000020CD
:105B10008380000070B505200121000700F010FF10
:105B200000240D4D002800D02C6002210B4800F00D
:105B300007FF002808D10A482C6000880A21484342
:105B40000849088003F0B0FF012000F031FE022078
:105B500000F02EFE70BD0000F00000200004005098
:105B6000CE000020DE0000207047000010B508497C
:105B700000224A6107494B684C1523434B604B6830
:105B8000082423434B60C009C001026010BD00001F
:105B900084160020002002407FB500250C460646F2
:105BA000039500F0D5FDE009029003A90196009548
:105BB000684600F065FD002804D000F09DFD00203F
:105BC00004B070BD00F098FD0120F9E710B5002386
:105BD00002E0C45CCC545B1C9342FAD310BD0000BD
:105BE00010B5214A00219069C305204804D54169B8
:105BF000022319434161911593699B0505D54369BA
:105C00000124234343616302194393695B0505D56E
:105C10004369082423434361E301194393691B0546
:105C200005D54369042423434361630219439369FF
:105C30009B0405D543691024234343616302194340
:105C400093699B0304D5446920231C434461194391
:105C50009369DB0305D54369402423434361A002D4
:105C60000143916110BD0000002002408416002015
:105C700070B5054600F070FE0646184C0AE0681C38
:105C800008D0002D04D000F067FE801BA84201D987
:105C9000032070BDA069C007F1D1A069800701D5BC
:105CA0000220A061A069C00511D4A06980050ED4AE
:105CB000A06940050BD4A069000508D4A069800440
:105CC00005D4A069800302D4A069C00303D5FFF7FF
:105CD00087FF012070BD002070BD00000020024041
:105CE000F8B51746002605460C4600F031FD09E0E0
:105CF00029460220226800F00DFD002804D1241D51
:105D00002D1D361DBE42F3D300F0F6FCBE4201D27B
:105D10000020F8BD0120F8BD10B50849024600205A
:105D2000054B497905E044001C5B944203D0401CBC
:105D3000C0B28842F7D310BD6E1200204800002088
:105D400010B5094800F0C6FF80B2FFF797FC074A7C
:105D5000074BFFF78DFB0022064BFFF7F1FBFFF728
:105D6000D3FC80B210BD0000B0140020F853E3A5AE
:105D70009B843E4000408F40F8B5414CE0790028BC
:105D800001D0002000E00120E0713D493D48CA7982
:105D90000275097A41753C490A780276497841765C
:105DA0003A48017837481330017005214172962036
:105DB00004F016FC4B20C00004F02CFC31490022FA
:105DC00013310C2004F0F6FC00210C2004F004FD3B
:105DD000022004F055FC2E4D00210F2004F07AFB28
:105DE0002842E062F8D0E06A411C3BD0294E2A4F9D
:105DF000400439D58122D20100210F2004F0AFFCEC
:105E00000021102004F066FB41061E48490E0022C6
:105E1000633004F095FB1B4D6335687A052820D16B
:105E200002221949681DFFF7CDF9002819D1A87A77
:105E3000607113480422691C4030FFF79FF9206C01
:105E400000F02EF860836079294642000B31084645
:105E50007330FFF793F9608B318848433880022014
:105E60002070F8BD02F058FC0C480188608B054694
:105E7000FFF73EF93088414339806D1E6583F8BDD8
:105E8000480000208D110020E0000020BE0000200E
:105E900000D02724C8000020C6000020CA0000202F
:105EA00010B504460E4800F015FF0E49C006C00E9E
:105EB000098805E02246C240D2070FD0401CC0B27C
:105EC0008842F7D3012005E02246C240D20705D020
:105ED000401CC0B28842F7D3491EC8B210BD0000B2
:105EE000B0140020CA00002010B5084800F096FA4F
:105EF0000A21064800F032FA044800F01DF9800536
:105F000003D5024800F01AF980B210BD54140020E5
:105F1000F8B52F4D00220121284600F016FDFFF7AD
:105F2000E3FFFFF790FB2B4E3146FFF7B1F92A4C08
:105F30000122A0601146284600F007FD2749A0680D
:105F4000002588423EDB2078254F002815D025709B
:105F5000FFF7CAFFFFF777FB3146FFF799F9A0601B
:105F6000FFF7F0FB00223B46FFF774FA00221D4BBF
:105F7000FFF77EFAFFF7FAFB6060A068FFF7E2FB2D
:105F800000223B46FFF766FA174A184BFFF770FAF4
:105F900006460F466068FFF7D5FB134A144B524282
:105FA000FFF766FA32463B46FFF7B0F9FFF7DEFB34
:105FB00010496060884201DD616004E0FF21C9058D
:105FC000C84200D365606068FFF766FBC0B2F8BDE9
:105FD0000004005000401B442400002000006040EA
:105FE00000000C4000E064403333333333B33040BF
:105FF000CCCCEC3F0000C842F8B50546044640351D
:10600000287C0026012808D0012028742068816897
:106010008907890F01290ED101E00220F8BD01682E
:10602000C90708D0606D2021084360650126002063
:1060300028743046F8BD616DFF220132914302227F
:1060400011436165C1688907890F0091C16889089A
:106050008900C1602068816892071143816000F067
:106060007BFC07460EE000F077FCC01B0A2809D92C
:10607000606D022188431021084360650020287468
:106080000120F8BD206880680028ECDB2068C1682A
:10609000009A1143C160606D80088000401C6065FB
:1060A000C5E70000F8B506460D464036317C0129AB
:1060B0000DD00121317401688A68520709D5416DFC
:1060C000202211434165002030740120F8BD0220D8
:1060D000F8BD174B6A68D80547109A42154C8A6A72
:1060E0002B6812D05B035B0B1A438A622968490351
:1060F00005D5A1680143A1600A20FFF757FC286875
:10610000800312D5A06838430EE05B035B0B9A4313
:106110008A622968490302D5A1688143A160286881
:10612000800302D5A068B843A06000203074F8BD99
:106130000110000000270140406D70470068006CAE
:106140007047000070B5040006D0606D264600253B
:106150004036002802D006E0012070BDA5653574E8
:10616000204600F0D3F8606DC00603D4216888682B
:10617000400705D5606D1021084360653574EBE775
:10618000606DFF22013290430222104360658868EF
:106190008207920F5B48012A02D10A68D2072BD1ED
:1061A000032362689B079A4205D05B429A4202D061
:1061B0005B009A4209D10A69920092080A6121683B
:1061C0000A6963681A430A610CE00A69920092083E
:1061D0000A6181680F22920491438160816862683C
:1061E000114381602168CA6818239A43CA602168F4
:1061F000CA68A3681A43CA608168012252069143A3
:1062000081608168A28E5206114381602068816896
:10621000C90004D4816801221207114381602068FB
:10622000C168394A1140C1602069E168022825D05F
:1062300000200143204620300278037B52035B009C
:106240001A431143226B1143A26992031143E2697D
:10625000D20311432268D3681943D160616A0A46A8
:10626000FF3AC23A05D0A26A11432268D3681943A3
:10627000D16042780121012A02D00BE00420D8E746
:106280000078002823D0606D202210436065A06D47
:106290000843A065E06B012820681FD00169C90789
:1062A00003D0016949084900016120684169C908B2
:1062B000C900416120684169A26B11434161A56534
:1062C000606D80088000401C6065002070BD206803
:1062D000C26801231B041A43C260DBE70269FF2383
:1062E0009B009A43026120680269236CA66C1A43E2
:1062F000636C33431A430261206802690A430261F6
:10630000D3E70000002701401902FEFF10B586B058
:10631000044614216846FEF74AFF0E492068884269
:1063200016D10D48416B421511434163C16A0122E8
:106330001143C162C06A6946104005900220009076
:1063400003200190002002900520000700F03CFA95
:1063500006B010BD0024014000100240F8B504460C
:106360004069254640350E4608280BD02068C06895
:10637000C00709D0606D20210843606500202874A3
:106380000120F8BD082700E00C2700F0E5FA009096
:1063900011E0701C0FD0002E05D000F0DDFA00993E
:1063A000401AB04207D9606D04210843606500209F
:1063B00028740320F8BD206800683842E9D0606D79
:1063C00001214902084360652068C16809058A0FF8
:1063D0000C21002A1BD12022125D002A17D102684D
:1063E000120714D5826853070122002B08DB43688B
:1063F0008B434360606D130298431043606506E071
:10640000606D202318436065A06D1043A065A069EE
:10641000002801D1206801600020F8BD70B5044655
:10642000216800208968490721D425464035297C08
:1064300001291CD001212974E169012904D02046D9
:10644000FFF7C6FA002811D1616D0A4A1140FF22F8
:106450000132114361650021A165297422681C2164
:10646000116021688A6804231A438A6070BD022083
:1064700070BD0000FEF1FFFF70B500240146203121
:106480004A79022A03D00421C163012418E002687A
:1064900013680E25AB431360026813685B085B004A
:1064A0001360436C1C221340012215469D40036C6F
:1064B0005D604A7100220A71816B002900D0884713
:1064C000204670BDF0B4016C0D6801680C68466C24
:1064D0001C2304221E401746B7402F420ED06707E8
:1064E0000CD50C68A40602D40C6894430C60416C73
:1064F00019408A40016C4A60016B1AE00227B740DC
:1065000002462F402032002F17D0A70715D50C6860
:10651000A40605D40C680A25AC430C600121517116
:10652000446C02211C40036CA14059600021117190
:10653000C16A002918D0F0BC08470827B7402F428D
:1065400012D0240710D50C680E25AC430C60446CA7
:1065500001211C400B46A340046C6360C163517170
:1065600000211171416BE4E7F0BC704770B5040085
:106570003CD01F48256814212818FEF7B9FD80007B
:1065800060641C482064022120462030024641718C
:1065900029681948E3680140A068666918432369BF
:1065A00033431843A3691843E3691843236A184324
:1065B000084328600121A0688903884210D00D4853
:1065C0008030836A656C1C210D400F26AE40B343BA
:1065D0008362656C63680D40816AAB400B438362E4
:1065E0000020E06301215171107170BD012070BD68
:1065F000F8FFFDBF000002400F80FFFFF8B5044622
:106600008C46203001790025012909D00126067128
:1066100041790027012905D0077102252846F8BDD8
:106620000220F8BD02214171E76320680168490832
:106630004900016061462046FFF716FA206B0028EA
:106640002068016801D00E2205E004229143016018
:10665000206801680A221143016020680168314303
:106660000160DBE770B5044600F076F90546601C72
:1066700000D0641C00F070F9401BA042FAD370BD3A
:10668000F8B51A4E0546307C0F46012807D0012088
:1066900030741748FFF7ECFA010002D021E0022025
:1066A000F8BD0020C04338606C6814E02046FFF756
:1066B0005DFA0F48FFF7DCFA01460E4842680823EE
:1066C0009A434260426843159A434260002901D0D0
:1066D0003C6006E08034A8686A68C0018018A04267
:1066E000E4D8002030740846F8BD0000841600206D
:1066F00050C30000002002400548416802221143B7
:106700004160416801221143416000207047000050
:1067100000200240F8B50C4C1646207C0F4601289C
:1067200008D0012020740948FFF7A2FA00250028AC
:1067300002D006E00220F8BD65613E600348FFF725
:1067400097FA2574F8BD00008416002050C300009D
:1067500011484168C9070BD0EFF3108172B60F4A98
:10676000C2600F4AC26081F310884168C9070ED128
:10677000416889070DD5EFF3108172B6094A0261AD
:10678000094A026181F310884068800701D5012021
:10679000704700207047000000200240EFCDAB8919
:1067A00005040302BFAE9D8C16151413704700003C
:1067B00010B504494A69024202D04861FFF7F6FF6A
:1067C00010BD000000040140F8B500230124A2E040
:1067D00027469F403A4070D04D68022D01D0122DBF
:1067E00014D1DD08AD002D1800952D6A5E07AC466A
:1067F000F50E0F26AE46AE406546B543AC460E6973
:106800007546AE4065462E43009D2E624D68012DB3
:1068100005D0022D03D0112D01D0122D16D185687F
:106820000326AC465D00AE46AE406546B543AC4679
:10683000CE687546AE4065462E43866046680D7943
:10684000BE43ED06ED0F9D403543456006685F0091
:106850000325BD40AE46AE430D79B446AE07B60F34
:10686000BE4065462E430660C6687546AE438D68D9
:10687000BD403543C5604D68ED004BD5294D6E6B6D
:1068800026436E639E08284DB6007519AC46AD6868
:106890009E07360F0F27B740BD4305273F07B84275
:1068A00001D1002715E0214FB84201D1012710E0A6
:1068B0001F4FB84202D102270BE02BE01D4FB84218
:1068C00001D1032705E01C4FB84201D1052700E0A4
:1068D0000627B7402F436546AF60184D2E684F68B6
:1068E0009643FF0300D516432E606E684F689643AB
:1068F000BF0300D516436E60AE684F689643FF0233
:1069000000D51643AE60EE684F689643BF0200D5CF
:106910001643EE605B1C0A681546DD4000D057E761
:10692000F8BD0000001002400000014000040050CB
:1069300000080050000C0050001C005000040140F2
:106940000069084000D001207047002A01D0816111
:10695000704781627047000001480068704700007E
:10696000F400002002480168491C016070470000E3
:10697000F400002010B508480024016840221143AB
:106980000160204600F00AF8002801D0012401E04F
:1069900000F0CCF9204610BD0020024070B505463D
:1069A00009487D210024C9000068FEF7A1FB00F022
:1069B00061FE002801D0012404E000222946501E77
:1069C00000F0D4F9204670BDF800002070477047F1
:1069D000F8B53A4C01266078401C6070E670208C57
:1069E000401C2084608902F099FB354FF888FEF73F
:1069F0002AFE3449FEF74CFC334D00902968FEF71F
:106A0000EEFB2860A16AF005814203DB0098FEF7E7
:106A10003BFCA06202212D48FFF792FF002808D01E
:106A20000020E0622A492F682A488F4227DD06703D
:106A300027E0F888FEF707FE2249FEF729FCE16A05
:106A4000FEF7CDFB2449E0628842EBDBE0790028C9
:106A500013D000211A484030818004F031F8012120
:106A6000002289021948FFF770FF7D200001FFF71F
:106A7000F9FD1B491948C860D4E70121EAE7002164
:106A80000170207A401EFEF7D3FD3946FEF78AFEDC
:106A900006D82079002803D01248C1793143C1714A
:106AA000207AFEF7D0FD2968FEF77CFE04D220791B
:106AB000002801D003F068FFF8BD0000BC000020F2
:106AC0002C0D002000007A44F0000020000400504B
:106AD000000040404E0000200000A0400400FA05E5
:106AE00000ED00E0A0110020704770B505000DD04A
:106AF00002202C462034A073284601F0E9FB2846EA
:106B000000F0BEF80020A073607370BD012070BD5E
:106B10007047704710B5044600680168C943C9074B
:106B200008D18168C943C90704D1012141602046C9
:106B3000FFF74EFF20680168C943890708D48168C0
:106B4000C943890704D4022141602046FFF73EFF74
:106B500020680168C943490708D48168C9434907C7
:106B600004D404214160204600F0DEF8206801686A
:106B7000C943090708D48168C943090704D4082117
:106B800041602046FFF7B0FF20680168C943C9068D
:106B900008D48168C943C90604D410214160204645
:106BA000FFF715FF20680168C943890608D481688A
:106BB000C943890604D4202141602046FFF7A9FF7C
:106BC00020680168C943490608D48168C943490659
:106BD00004D4402141602046FFF79AFF10BD000019
:106BE000F8B5040005D025462035A87B002802D042
:106BF00006E00120F8BD00206873204600F052F83E
:106C00000220A8732068C26884466368012B04D000
:106C10000120A16AC005814201D11E20824315488E
:106C20006169814201D0144802401448A6680240BC
:106C300018463043676A266A3E433043A66A3043AB
:106C40001043012B03D00122D205964203D12369C0
:106C5000E2681A431043074A914205D0A2691143E2
:106C6000E2690243084610436146C8600120A873E8
:106C70000020F8BDFFFF00003F1FFFFFF8F119FFE4
:106C800010B500680549884207D10548816B490065
:106C9000490881630D2000F055F810BD007C0040CC
:106CA0000010024010B50068084988420CD108481D
:106CB000816BC20411438163002201210D2000F089
:106CC00055F80D2000F048F810BD0000007C004091
:106CD000001002400068C0697047000070B50224CF
:106CE000034620339C730F4C2568E604354325602A
:106CF0000468E568B6123543E5600568AE680124AE
:106D00002643AE6005682E6926432E610568A96199
:106D100001684A61006801690422114301619C73A2
:106D2000002070BD00040140704700000448416B22
:106D3000012211434163816B020411438163704757
:106D400000100240C106C90E0120884001490860B8
:106D50007047000080E100E0C106C90E01208840B4
:106D6000014908607047000000E100E010B501F043
:106D7000B1FC10BD02494A6882434A607047000076
:106D8000007000400248016882151143016070479D
:106D90000070004002494A6802434A6070470000A0
:106DA0000070004005480168022211430160044858
:106DB000016904221143016130BF70470070004037
:106DC00000ED00E00A4B1A689208920002431A6034
:106DD00008480369042213430361012906D040BF18
:106DE00020BF20BF016991430161704730BFF9E7BF
:106DF0000070004000ED00E0F8B504460078544D06
:106E0000800672D5524E0027403EB06BC00004D4BD
:106E1000B06BA9050843B06301274E480168C90556
:106E200011D40168821511430160FFF795FD0090B0
:106E300005E0FFF791FD0099401A642837D84548CE
:106E40000068C005F5D532680321090560680A406D
:106E50000140914208D08103890F032904D1316890
:106E6000890301D50120F8BD2A69032109040A40DC
:106E700022D0084090421FD0207880061CD5286977
:106E80002A6988430121C9040A432A612A698A437D
:106E90002A612861C0050FD5FFF75EFD009008E06C
:106EA000FFF75AFD0099411A2B48814201D903206E
:106EB000F8BD28698005F3D561688803800F032831
:106EC00005D132680005824301400A4332602869D7
:106ED000032261681204114008432861002F04D086
:106EE000B16B012000078143B1632078C00705D052
:106EF000E868A168800880000843E860207880077F
:106F000005D5E8680C218843E1680843E8602078EB
:106F1000400706D5E86803218902884321690843B0
:106F2000E8602078000706D5E86803210903884354
:106F300061690843E8602078000606D5E868032107
:106F400089048843A1690843E8600020F8BD000077
:106F5000401002400070004088130000F8B50E4653
:106F600005007DD053480068C007C00FB0420AD268
:106F70005048016849084900314301600068C00772
:106F8000C00FB04271D128784B4C800705D5E0681E
:106F9000F0218843A9680843E0602878C00752D0F0
:106FA0006868022817D0032818D02168012818D053
:106FB0008905002959DAE168890889000143E160FF
:106FC000FFF7CAFC69680746022912D003291CD0C2
:106FD000012926D033E021688903EAE72168890185
:106FE000E7E74907E5E7FFF7B7FCC11B33488142F4
:106FF00023D8E0680007800F0228F4D123E0FFF7D0
:10700000ABFCC11B2D48814217D8E0680007800FF8
:107010000328F4D117E0FFF79FFCC11B27488142EA
:107020000BD8E0680007800F0128F4D10BE0FFF7D0
:1070300093FCC11B2148814201D90320F8BDE068BF
:107040000007800FF3D11B480168C907C90FB1427F
:107050000DD901684908490031430160006800E02A
:1070600003E0C007C00FB04201D00120F8BD28786E
:10707000400706D5E068072109028843E96808430C
:10708000E0602878000707D5E0680721C902884337
:107090002969C9000843E06000F036F8E168084A51
:1070A0000906090F515CC840064908600020FFF737
:1070B00075FCF8BD0020024000100240881300005B
:1070C000BEAB0008F8000020044805490068C96804
:1070D000044A4905490F515CC8407047F800002038
:1070E00000100240D7AB0008044805490068C96891
:1070F000044A8904490F515CC8407047F8000020D9
:1071000000100240D7AB000810B5184AD1680C2017
:10711000084004280BD0082810D00C2810D0506844
:107120000004410F0120C003491C884010BD1068B5
:10713000C00601D50E4810BD0E4810BD0E4810BD4A
:1071400088020E4B000F185C0902D368890F491C96
:10715000DB0301D5084A05E01268D20601D5044ACE
:1071600000E0044A5043FDF7C3FF10BD0010024089
:1071700000093D000024F40000127A00CEAB0008A4
:10718000FEB505007ED0FE4CE7680C20E66807409F
:107190000120000406402878C00747D0082F05D0FA
:1071A0000C2F0AD101200004864206D120688003FA
:1071B0003CD568680028E5D038E001206968000403
:1071C000814203D121680143216011E0052301229E
:1071D0001B0492049942216802D111432160F1E716
:1071E0008143216021680140009120689043206024
:1071F000686800280DD0FFF7AFFB009005E0FFF7AF
:10720000ABFB0099401A64287AD820688003F6D531
:107210000CE0FFF7A1FB009005E0FFF79DFB009954
:10722000401A6428F0D820688003F6D428788007B4
:1072300055D50923E868042F0DD00C2F01D1002E5D
:1072400009D000283BD02168994301432160FFF712
:1072500083FB064627E02168490701D5002891D025
:1072600061681F22120291432A6912021143616070
:107270002168994301432160FFF746FFE168090651
:107280000A0F00E079E1BF49895CC840BE49086047
:107290000020FFF783FB002872D120E0FFF75CFBA2
:1072A000801B0228B0D820684007F7D560681F21EE
:1072B0000902884329690902084360600FE02068D9
:1072C000400840002060FFF747FB064604E0FFF758
:1072D00043FB801B022897D820684007F7D4287802
:1072E000C0065FD5002F0CD0A869002849D02068BF
:1072F000FF21013108432060FFF72EFB06462DE0F9
:10730000C0E02068800502D5A8690028A7D0606881
:10731000072149038843296A084360606068297F20
:107320000002000A090608436060286A410B012038
:10733000C003491C8840E16809060A0F9149895C2D
:10734000C840914908600020FFF728FB002817D1AA
:1073500028E0FFF701FB801B0228A3D820688005E6
:10736000F7D56068072149038843296A08436060AC
:107370006068297F0002000A09060843606011E086
:10738000E1E02168FF20013081432160FFF7E4FA4A
:10739000064604E0FFF7E0FA801B022872D8206856
:1073A0008005F7D42878794E000724D5686900282D
:1073B000306910D0012108433061FFF7CDFA009009
:1073C00005E0FFF7C9FA0099401A02285AD8306937
:1073D0008007F6D50FE0400840003061FFF7BCFAA7
:1073E000009005E0FFF7B8FA0099401A022849D842
:1073F00030698007F6D42878400765D500200290D0
:10740000A06BC00006D4A06B012109070843A0634C
:10741000012002905E480168C90511D401688215F7
:1074200011430160FFF798FA009005E0FFF794FA26
:107430000099401A642825D855480068C005F5D53C
:10744000FF20AA680130824203D1316901433161D2
:1074500011E001218902002A07D005231B029A426C
:1074600003D132690A433261EFE732698243326104
:10747000306988433061A86800280FD0FFF76CFAA4
:10748000009007E05EE0FFF767FA0099411A414873
:10749000814257D830698005F5D50DE0FFF75CFAD9
:1074A000009006E0FFF758FA0099411A39488142E6
:1074B00048D830698005F5D40298002804D0A06B24
:1074C000012109078843A063686A002864D00C2F53
:1074D0003ED0012636060228206805D0B043206041
:1074E000FFF73AFA05462FE0B0432060FFF734FA81
:1074F000074604E0FFF730FAC01B022822D82068B4
:107500008001F7D4E96AA86AE2680843296BFD2381
:107510001B049A4311430843E06020683043206015
:10752000FFF71AFA054604E0FFF716FA401B022897
:1075300008D820688001F7D52EE0FFF70DFA401B30
:10754000022801D90320FEBD20688001F5D423E084
:107550000128F8D0E06801210904AA6A014091429B
:107560000BD10F218904EA6A0140914205D1032120
:1075700089050840296B88420ED00120FEBD00001D
:1075800000100240BEAB0008F8000020401002408E
:1075900000700040881300000020EFE770B5040081
:1075A00007D0002625464035A662687C002802D018
:1075B00005E0012070BD2E74204600F02FF8022057
:1075C000687420680168402291430160A168606886
:1075D00022690843E16811430843616901220843B5
:1075E000A169520211400843E1690843216A084336
:1075F000A16A084321680860A0690421000C0840C2
:10760000616A0843216848602068C169920091431B
:10761000C161666501206874002070BD10B586B038
:10762000044614216846FDF7C2FD104920688842CF
:1076300019D10F48416B821411434163C16A012281
:107640001143C162C06A002110400590E020009003
:1076500002200190032003900291049105206946C5
:107660000007FFF7B1F806B010BD00000030014080
:1076700000100240094910B5401E884201D901207E
:1076800010BD074C60610321081F01F023F80020A2
:10769000A06107202061002010BD0000FFFFFF0057
:1076A00000E000E0F0B502462032137E012B15D039
:1076B000012717760223537605686C68AB6870263D
:1076C000B4430E68496826438024A34319436E607F
:1076D00000688160577600201076F0BD0220F0BD72
:1076E00070B5040005D025462035687E002802D0FC
:1076F00006E0012070BD00202876204600F00AF840
:1077000002206876211D206801F0C2FD0120687604
:10771000002070BD006801218907884204D1034818
:10772000816B012211438163704700000010024009
:10773000F8B5054604462035287E012817D00126D5
:107740002E7602206876226890687727FF23B84358
:107750001B02984390600A68502A31D00EDC202A20
:107760004BD006DC002A48D0102A3AD145E002204E
:10777000F8BD302A41D0402A33D136E0602A27D0E4
:10778000702A12D001200003121A2AD0824228D176
:10779000CB684A688968206801F0B3FD2068816879
:1077A00001229203114381601BE0CB684A6889681B
:1077B000206801F0A6FD216888683843886010E0E1
:1077C000CA684968206801F016FE5021206806E06A
:1077D000CA684968206801F01FFE6021206801F036
:1077E0009BFD6E7600202876F8BDCA68496820683F
:1077F00001F001FE40212068F1E711462068EEE724
:1078000010B586B0044614216846FDF7D0FC01216E
:1078100020688907884212D10A49CA6A02200243B5
:10782000CA62C96A0190014005914102009100219C
:1078300002910391049069460348FEF7C5FF06B024
:1078400010BD00000010024000040050F8B50646CC
:1078500004462036307E0D4601280DD001203076BA
:10786000022070760427002A08D0042A16D0082A9D
:107870002AD00C2A4DD137E00220F8BD206801F053
:1078800053FD206881690822114381612068816964
:10789000B943816120688169EA6812E0206801F0DB
:1078A0005BFD206882690121C9020A438261206868
:1078B0008169012292029143816120688169EA68AD
:1078C00012021143816124E0206801F05EFD20680E
:1078D000C26908210A43C2612068C169B943C16114
:1078E0002068C169EA6812E0206801F069FD20683B
:1078F000C1690122D2021143C1612068C26901211C
:1079000089028A43C2612068C169EA681202114390
:10791000C1610120707600203076F8BD70B504009A
:1079200005D025462035687E002802D006E00120DB
:1079300070BD00202876204600F00AF80220687604
:10794000211D206801F0A4FC01206876002070BD94
:10795000704710B504460068012201F0C5FC20689C
:1079600081684907490F062903D0016801221143A4
:107970000160002010BD000010B504460068002220
:1079800001F0B2FC2068016A054A114203D1016886
:10799000490849000160012020346076002010BDB4
:1079A0001111000070477047F8B502680446D069AD
:1079B0001168936805072D0F5BD0DD07ED0FFF26DB
:1079C00021360E402E4367D0C60706D0CE0504D51B
:1079D00001261662E26F3243E2678707022204261D
:1079E000002F06DADF0704D027683A62E76F3743D3
:1079F000E767470706D5DB0704D023681E62E36FFD
:107A00001343E367020709D520220A402A4305D021
:107A1000236808221A62E36F1343E367E26F002AC8
:107A20002FD0800606D5880604D5216E002901D006
:107A300020468847E06F21688968490601D400071D
:107A400024D5204601F08EFE20688168490619D5AC
:107A50008168402291438160E06E002812D0204965
:107A60008163E06EFEF708FD00280AD0E06E816BAE
:107A700006E0850610D58D060ED5216E1CE0204649
:107A80008847F8BD2046FFF78EFFF8BD2046FFF778
:107A90008AFF0020E067F8BDC50208D55B0206D565
:107AA0000120000510622046FFF77CFFF8BD0306A9
:107AB00005D50B0603D5616E0029E0D1F8BD40065F
:107AC000FCD54806FAD51368204640218B43136045
:107AD000202161670021616600F069F9F8BD0000AE
:107AE000C196000810B5040003D0606F002802D0D2
:107AF00007E0012010BD002170200155204600F054
:107B000027F824206067206801684908490001605F
:107B1000204601F071FE0128ECD0606A002802D0F6
:107B2000204601F0AFFC206841680922D20291434F
:107B30004160206881682A22914381602068016841
:107B4000012211430160204601F002FD10BD00003A
:107B5000F0B587B0064614216846FDF728FB2C498E
:107B60003068884251D12B48416B01229203114366
:107B70004163C16A01221143C162C06A00251040FD
:107B800005900320400200900220032701A9A1C113
:107B900004200490052069460007FEF715FE1F4CDF
:107BA0001D48A560E56081C48027E560A7602020AE
:107BB000256160610002A0611848083CFEF7D6FC10
:107BC000002801D0FDF7D0FFF466A662144C1248DD
:107BD0002146143820600320606010200831A1C1C4
:107BE0006561A561E56120462562FEF7BFFC0028BE
:107BF00001D0FDF7B9FFB466002201211B20A66267
:107C0000FFF7B4F81B20FFF7A7F807B0F0BD00009E
:107C1000003801400010024030000240F4150020FE
:107C20003C160020F8B50446806F20284DD100296D
:107C30000BD0002A09D00123A0681B03984206D16B
:107C40002069002803D1C80701D00120F8BD2546CE
:107C50006035287C012838D00120287458206165BF
:107C600002530026E6672220A067E06E002819D0A4
:107C70001749C162E16E17480863E16E1648486310
:107C8000E06E13468663676D21683A462431E06EE4
:107C9000FEF7B4FC002805D01020E0672E742020E9
:107CA0006067D2E72E7420680168FF220132114319
:107CB0000160206881680122114381602068816829
:107CC0004022114381600020F8BD0220F8BD000071
:107CD0001D9700085B970008D5960008704770470D
:107CE000FFB50446406F83B017460D4620285CD18F
:107CF000002D0AD0002F08D0A168C001814207D111
:107D00002069002804D1E80702D0012007B0F0BDA7
:107D1000204660300290007C012846D00298012164
:107D200001740020E06721206067FEF715FE2646FB
:107D300040360190378277820120A168000381429A
:107D400002D12069002802D02F46002511E000272B
:107D50000FE000228021204601F062FE002815D1AC
:107D6000002F15D02168387888627F1C708A401EE9
:107D70007082708A019B002806980090E9D1002249
:107D80004021204601F04CFE002808D00320BDE72A
:107D900028882168C005C00D8862AD1CE6E7202058
:107DA0006067029900200874B0E70220AEE77047D0
:107DB00001490248C160FDE70400FA0500ED00E05A
:107DC00070B586B014216846FDF7F1F90F4801241B
:107DD000818B002900D18483808B012805D0022863
:107DE00001D100F0FFFB06B070BD0122084E9502E4
:107DF00029463046FEF7A9FD002102910391009526
:107E0000019469463046FEF7DFFCECE7BC00002039
:107E10000004005070B501240E4DA4030022214639
:107E20002846FEF792FD002204212846FEF78DFD2C
:107E30000A2002F0F2F8012221462846FEF785FDCD
:107E40000A2002F0EAF8002221462846FEF77DFDCE
:107E500070BD00000004005070B501240E4DA40355
:107E6000002221462846FEF770FD01220421284603
:107E7000FEF76BFD0A2002F0D0F8012221462846C9
:107E8000FEF763FD0A2002F0C8F8002221462846CA
:107E9000FEF75BFD70BD000000040050F1B500244A
:107EA0000126154F2546B603002231463846FEF717
:107EB0004CFD0A2002F0B1F8012231463846FEF7A7
:107EC00044FD6006040E04213846FEF739FD002803
:107ED00001D0641CE4B2052002F09FF86D1CEDB2E5
:107EE000082DE1D30098002803D0FFF793FF204628
:107EF000F8BDFFF7B1FFFAE700040050F8B501261E
:107F0000154F0546B603002231463846FEF71DFDE3
:107F10000024E80901D0012200E0002204213846B3
:107F2000FEF713FD6806050E0A2002F076F801221E
:107F300031463846FEF709FD0A2002F06EF80022AD
:107F400031463846FEF701FD0A2002F066F8641C4F
:107F5000E4B2082CDDD3F8BD0004005070B50D4C20
:107F6000012204212046FEF7F0FC01229503294658
:107F70002046FEF7EAFC002204212046FEF7E5FC3D
:107F80000A2002F04AF8002229462046FEF7DDFCCE
:107F900070BD00000004005070B501240E4DA40314
:107FA000002221462846FEF7D0FC00220421284664
:107FB000FEF7CBFC0A2002F030F8012221462846C9
:107FC000FEF7C3FC012204212846FEF7BEFC0A206E
:107FD00002F023F870BD00000004005070B5144D8D
:107FE0000024012204212846FEF7AFFC062002F0FF
:107FF00014F80122960331462846FEF7A6FC062017
:1080000002F00BF807E0641CE4B2FA2C03D9FFF786
:10801000C3FF012070BD04212846FEF791FC002813
:10802000F1D1002231462846FEF78FFC002070BDBA
:1080300000040050F8B501F0BBFA01F0F5FA55481C
:108040000068C069544E554F800700D5FE60FDF7AB
:1080500077FE5349534D898F534C002929D05349FA
:108060000A7801218902002A05D0012A0ED0022AAD
:1080700010D0032A1DD1A08B01282CD0022818D1A2
:10808000444808213C38FFF777FC12E0FF22F53224
:108090009042F0D2A08B01281BD0022804D008E027
:1080A0002846FEF752FC04E03A4808213C38FFF726
:1080B00050FC40213B48FEF743FC002500282CD013
:1080C0003B480560FDF724FF2070A079002804D00C
:1080D00007E00022E4E70122E2E70120A07101F0BD
:1080E000E3FC2078632806D9002208212D48FEF7FA
:1080F0002CFC012205E0012208212A48FEF725FC7C
:10810000002201210520C9030007FEF71EFC244CB4
:108110004034A08C012803D01CE0A5710022EBE7BD
:1081200024486946088072B680212348FDF734FD53
:10813000002804D0022269461F48FDF7D1FD62B62F
:108140001EA001F04DFDA58402F0BAFC642001F0F0
:108150005DFFFE60608C012808D1114865840580B0
:1081600002F0AEFC642001F051FFFE60208C01287B
:1081700006D1258402F0A4FC642001F047FFFE60D4
:108180000748124A0188914202D1C088002800D1D4
:10819000FE60F8BD741500200400FA0500ED00E053
:1081A0002C0D002000040050BC0000205A000020CC
:1081B000F0000020AAAA0000384A0008BDF8C8EB69
:1081C000C9FDBCB6C4A3CABD0D0A0000AA55000073
:1081D00008B53721202000F06EF80321212000F09F
:1081E0006AF84021222000F066F80821232000F0E0
:1081F00062F8AA21302000F05EF80A4802210187C7
:10820000322000F058F80121332000F054F85F21AB
:10821000202000F050F8684600F006F80A2001F02F
:10822000FCFE08BD2C0D002010B501460F2000F00B
:1082300021F8002800D0012010BD10B50446FFF73A
:108240008DFE3220FFF75AFEFFF7C8FEE0B2FFF7BF
:1082500055FEFFF7C3FEFFF781FE3320FFF74EFE0A
:10826000FFF7BCFE0020FFF719FE0446FFF794FE5F
:10827000204610BD10B50C46FFF7DFFF207001202F
:1082800010BD70B50D460446FFF768FE3220FFF7BB
:1082900035FEFFF7A3FEE0B2FFF730FEFFF79EFECC
:1082A0002846FFF72BFEFFF799FEFFF775FE0A2021
:1082B00001F0B3FE70BD10B5FFF7E3FF012010BD64
:1082C00010B50248FEF726FC10BD0000B0140020D7
:1082D000FEB50446002572B60068394A831804D1F9
:1082E0003849CD68032189040D4081680191C16836
:1082F000009141698669002B08D132484038836A71
:10830000C7043B438362836ABB43836208463043AE
:1083100048D02B482368C34205D12A48C3680322AA
:1083200092049343C360002917D020680269012397
:108330001A43026120684161FEF70EFB0746FEF713
:108340000BFB2168C01B0968090703D47D21C90004
:108350008842F4D9216808204860002E17D0206890
:10836000016901221143016120688661FEF7F4FA78
:108370007D270646FF00FEF7EFFA2168801B09689B
:10838000C90601D4B842F6D92168102048600C48CB
:108390002168C14206D10B48C1680322920491436F
:1083A0002943C160206801694908490001612168C9
:1083B0000198886021680098C86062B6FEBD000020
:1083C0000084FFBF401002401CB5002116480091F8
:1083D000144A01910260C163120542608160072264
:1083E0008263012202610246C16020321170FF23C4
:1083F0005170C2334362816211730163816104224F
:1084000041634261C161FDF79DFE08480090801301
:10841000019069460448FDF745FE00210248FDF73A
:10842000EBFD1CBD00240140541400200200000498
:1084300008B50848016B012211430163006B01215B
:108440001040009000220A20FEF790FC0A20FEF760
:1084500083FC08BD00100240F0B587B014216846C7
:10846000FCF7A5FE4648C26A04210A43C262C26AFA
:108470000A400592C16A80263143C162C16A314017
:108480000591C16A01242143C162C16A214005915D
:10849000C16A02252943C162C06A2246284005906C
:1084A000052010210007FEF750FA01223549364811
:1084B000FEF74BFA002235493348FEF746FA912180
:1084C0000520002209020007FEF73FFA304801901C
:1084D000002705206946029700940007FEF774F90B
:1084E0002C480090112001900320039002976946C8
:1084F0002548FEF769F910206A46039591C20520C8
:1085000069460007FEF760F911200190029769465D
:10851000039700941C48FEF757F91F4801906946DD
:10852000009502941848FEF74FF9402000906946E4
:10853000019702951448FEF747F91848694691C11A
:10854000694611480397FEF73FF9912000026946FA
:1085500091C10520694600070397FEF735F9694682
:108560000948019700960294FEF72EF90022012196
:108570000520FEF7FBFB0520FEF7EEFB07B0F0BD84
:1085800000100240054200000004005008300000C6
:10859000000011100440000000002110083200000B
:1085A00010B50F4C0D482060FF20053060600020A2
:1085B000A060E06020616061E06101212062490209
:1085C0006062A161A0620720E0622046FEF7E6FF3C
:1085D0002068016840221143016010BD0030014055
:1085E000E014002010B58AB0002404940594069489
:1085F0000794089401211848099400940194029466
:108600008907039401600921846041600461134972
:108610004461C160FFF764F801200003049004A9DD
:108620000D48FFF785F80C48FFF778F9089408A97A
:1086300009480994FFF736F8602000900848019037
:1086400002940822694603940348FFF7FFF80248A2
:10865000FFF7D6F80AB010BD3815002093040000CB
:108660005702000000B585B014216846FCF79FFD55
:10867000164815490160E1214902416000218160ED
:10868000C160016181610C22C161426101623021DE
:1086900041620121090381634900C163FFF722FAA6
:1086A000012080020090022001900120029003200E
:1086B000039004200490052069460007FEF784F823
:1086C00001F0ECF905B000BD003801407415002040
:1086D000704700008307FF22DB0E9A408907090ECE
:1086E000994000280BDA0007000F08388308084873
:1086F0009B001818C36993430B43C36170478308F9
:1087000004489B001B181868904308431860704782
:1087100000ED00E000E400E0BFF34F8F04490348A0
:10872000C860BFF34F8F00BFFDE700000400FA05EB
:1087300000ED00E0F0B58FB0962001F051FF4B2026
:10874000C00001F067FFFF4C00256570A07B0C287E
:1087500001D30B20A0730122052051020007FEF770
:10876000F4F8A07B60736071F748A570F74E00784D
:108770003070F748022100783071F648FEF7E0F8D3
:10878000002862D00020A179F04E49000843F07122
:10879000A06AF070401CA06260793146B07242005D
:1087A000CE310846C338FCF7E9FC0620707230462B
:1087B00013380290217F0175617F41756079002235
:1087C000400031460D3001F0F5FF60790021400096
:1087D0000D3002F001F8022001F052FFF57125740E
:1087E000A57201202073E572DB48FEF773FA20843E
:1087F0000646A5706079FCF741FFD84AD84BFCF7D4
:1088000037FE01F09FFB0022D64BFCF77FFDFCF703
:108810007BFF0006C10C881980B20121C903608466
:10882000884201D3401A6084CF486063E078401CDE
:10883000E070C948FEF74EFAE083CC480C90C3487C
:108840004E300B901630019027E201209BE7C24882
:10885000FEF740FAE083C64EC64F21E0A07A00281A
:1088600013D001F07EFE039988420ED90699884202
:108870000BD201F04DFD2573099801F0AAFE0120ED
:1088800001F0FEFE2072A57211E0B348FEF722FA55
:1088900080B2E083618C884202D3C919884206D332
:1088A00000210F2001F016FE3042E062D6D0E06ACF
:1088B000411C1FD040047DD58122D20100210F2010
:1088C00001F04DFF0021102001F004FE41069F48F9
:1088D000490E002250300A9101F032FE002001F0D2
:1088E00099FE002001F04BFE984E5036707A072812
:1088F000AAD101E0FFF710FF02229F49701DFCF78B
:1089000061FC0028A0D19148503001788E48007851
:10891000814299D100273E460DA801F028FE04208F
:108920000DAA390E36020E433902175C0F43401E62
:10893000F7D5A764E66400273E46104601F009FE1D
:1089400004200DA93A0E360216433A020F5C174373
:10895000401EF7D527656665A1786A46491CA17057
:108960007A494D310E7916774F7969464F77607B9A
:10897000002809D1012275482271898BCE300180EF
:10898000627102980675477570486946CE30008856
:10899000898B059188427DD10B987849008A08809F
:1089A0006A4826464C30808A20836B48FEF792F94D
:1089B000F08300E066E1308B7149FF30C33080B254
:1089C000308388420CD9494240186C49308308886A
:1089D0006B4A401C80B20B320880904200D30D805D
:1089E0006849032008700B98564A81891186C0890E
:1089F000644B5086903B326B1A601A46B03AD37C77
:108A00001F073F0F032F00D0B7741A09F274F570D7
:108A100001274C4AB7729186D0867079FF21913137
:108A200048435749326D593940180104C817736DCE
:108A3000891858410206080A104353490990401802
:108A40000390192109988902401806900998B843A3
:108A5000010E0002F165B0653C48F36C0A30B26C5F
:108A600001F0E0FE3948736D1630326D01F0DAFE28
:108A70003648F36D1230B26D01F0D4FE3348082150
:108A80004172314900220978017070792F498000C4
:108A90001C3000E09EE001F08DFE70790021800026
:108AA0001C3001F099FE29492648F7720422513101
:108AB0004030FCF763FB3148318B07887D20C000D4
:108AC00078434018B0630D9030480078F073009000
:108AD00026484038C088FCF7B6FD05903846FCF7BC
:108AE000B2FD0599FCF7D4FB7F21C905FCF777FBA4
:108AF000FCF7D2FD81B2254801800098401E8142DA
:108B000001D10120F072B7841420305EFCF7A2FD81
:108B100007910890F08BFCF7B1FD1D4A1D4BFCF747
:108B2000A7FC00910A900D98FCF794FD009B0A9A0F
:108B3000FCF790FC079B089AFCF7E8FBFCF7C0FDEC
:108B4000F06329E048000020BE000020A0110020B2
:108B5000BC00002000040050B01400206666666669
:108B60006666E63F00000840A08601006C0D00200C
:108B700000D02724983A0000E0000020EC000020FC
:108B8000E70300003013002000AEFCFFDC000020F3
:108B9000F853E3A59B843E40BE48008800F0BEFA2F
:108BA000F07C002879D00C990988814275D00C9806
:108BB000E17C01801222B8480199FCF7DFFA082213
:108BC000B549B648FCF7DAFAB349B4480A22083185
:108BD000303057E10846FDF79FF8617B88420CD39F
:108BE0000122227162794300521C6271AA4A0599DE
:108BF000CE3AD15202990E754F75A74903220C390E
:108C00000A540B99A64A8B8913868700C989A24802
:108C100051869C38216BC151B038C27CA37C1107AE
:108C2000090F2646994202D9032900D0B274F17C7B
:108C3000002912D002229B49401DFCF7C3FA0028EC
:108C40000BD1012098493074C8710A981638C2B205
:108C5000727491480199FCF791FA9348736D381832
:108C60001630326D01F0DEFD7079002280008E49F1
:108C70001C3001F09FFD7079002180001C3001F054
:108C8000ABFD0AE0324600210F2001F068FD207B99
:108C9000002802D0002001F072FCE18B608C814240
:108CA00000D2D4E5814A80188142FAD880480188F0
:108CB00088000818E178884200D2A5747D4A002116
:108CC0000F2001F04CFDA0786071734800260C382D
:108CD0000078002812D1206CFDF7E2F807467648AC
:108CE00001883846FCF704FA74487F1E0088414327
:108CF00088B268490880678300F010FA0020A073EA
:108D0000617B22798A1822E0634B0C3B195C0029B5
:108D10001BD0A57BB3006D1CA5735F4D9C463C3DED
:108D2000E9505D4B4500CE3B77005D5B1833DD536A
:108D300085001A33584F5D5963466C3FFD50761CD1
:108D40003B466033491EF6B21954401CC0B2824201
:108D5000DAD8A078032801D2A07BA0735049002262
:108D6000887B48730390401E31E000212BE04A4C81
:108D70008B006C3CE6581D1906956D68AE4220DDEF
:108D8000B646454E4C00B63E365B9700B446424E62
:108D90003C3EF6590796404E6C3EF55035464A3DEE
:108DA00067197D884A3E355334467A341C197A3621
:108DB0006568F550069B76465E6066467E80079E37
:108DC0006660491CC9B28142D1DB521CD2B28242D8
:108DD000CBDB334800214172039C2BE02E4B2E4A03
:108DE000CE3B4F00B63AD25BDA531D468A0062355D
:108DF0001E46AD583236B550314EB54218D01D46DC
:108E00009235AD580A2D13D1457A0626AC467543E6
:108E10001E461A3EFB18AD191B88AB8033464C33F7
:108E2000D2181388EB8052882A8165466D1C4572E2
:108E3000491CC9B2A142D1D3174A0021204B9C3A08
:108E40008C00491CC9B213510C29F9D3007C0028AD
:108E500005D011490B7848788A78022B0ED0154A34
:108E6000002180320F2001F07AFC01210520002230
:108E700049020007FDF769FD0FB0F0BD074BC91CA3
:108E80009B1F1818FCF77AF901F01AFE642001F014
:108E9000BDF82FE5C60000203C130020320D002055
:108EA00048000020E0000020A0110020983A0000B7
:108EB000CE00002000D02724CA000020C8000020D7
:108EC000FFFF010070470000FEB5444942480860BA
:108ED00001F096FD424800F0E1F8424C2083404802
:108EE000801C00F0DBF860833D48001D00F0D6F8E0
:108EF000A083FF203C4D1D3068802846403001791A
:108F0000E1710291E88E3949C0B208700190E88F92
:108F10002071A88F6071A87AA070A8880090606204
:108F20002889FCF7ABFB324A324BFCF7A1FA01F07F
:108F300009F80022304BFCF7E9F9FCF7E5FB86B2B3
:108F4000A681EF8831463846FCF7D2F8E081014629
:108F50000098FCF7CDF871438EB27D20C000668189
:108F60007043FCF78BFB254A254BFCF7E9FAFCF72D
:108F7000CBFB20827D20A6823946C000FCF7B8F8E2
:108F80006082E083688F207202990120002902D15B
:108F900020710A212172002F01D16421E980019AF8
:108FA0001249432A01D943220A702084FCF7C8FEE3
:108FB000E082228A13491448FDF790FE13A0616AEB
:108FC00000F00EFEE98815A000F00AFE298918A01D
:108FD00000F006FEFEBD0000D59A00084400002007
:108FE000004F0008BC0000202C0D002000000020D5
:108FF000666666666666E63F00000840F853E3A5CD
:109000009B843E40FF7F0000B0140020B1EAC7A956
:1090100049443A202564202E0D0A0000CDA8D1B67F
:10902000BCE4B8F43A202564206D732E0D0A0000CC
:10903000B5A5B4CECDA8D1B6BBF9D5BECAFDC1BFCA
:109040003A202564B8F62E0D0A00000070B586B0EF
:1090500014216846FCF7ABF801250F4EED03002202
:1090600029463046FDF771FC01200024019002944E
:109070006946009503943046FDF7A6FB0320019056
:1090800002946946009503943046FDF79DFB02204B
:1090900000F0BCFF06B070BD0004005000887047AF
:1090A00070470000F8B5044600206A461080194D4C
:1090B00055222A70AA226A700322AA70661DEE70D9
:1090C0002A716971144A49008918AC712246E81D59
:1090D000FCF754F8002007E029186A4689781288BE
:1090E00089186A461180401CB042F5DB611DA81C3E
:1090F000FCF7A0FC01466846018029190078C87178
:1091000068464078087221460931024800F042FB67
:10911000F8BD0000F01300202C0D002010B51349FD
:109120000A8CCB8B9A4201D3D21A0A84104A098C3A
:10913000D2884A437D211018C90048430D49096867
:10914000401AFCF787FA0C4A0C4BFCF7F9F9FCF7CC
:10915000B7FA0B49884201DD4A428018002800DA3C
:10916000401808490968486110BD0000BC00002093
:109170002C0D002084000020F853E3A59B843E4082
:10918000FF7F0000B0140020034A1168382389B221
:1091900099430143116070470030014010B5FDF75D
:1091A000E1FB10BD10B59AB034216846FBF7FFFF14
:1091B00014210DA8FBF7FBFF1C2112A8FBF7F7FFFA
:1091C0001B4801680324E402A143C214891801600A
:1091D000FDF7D8FD17480169A14301610620009001
:1091E000FF20013002900120039010200490022003
:1091F000099040040B90000100240C900A946846EA
:10920000FDF7BEFF0F200D9003200E900F941094D9
:10921000012111940DA8FDF7A1FE812012900320D9
:1092200080041890149412A8FDF7E6FD1AB010BD42
:109230000070004040100240104801688215114340
:109240000160C1680E4A1140C16001680D4A1140B9
:109250000160816849084900816001680122920427
:1092600091430160C168FD2212049143C160002155
:109270000161064904488860704700000010024000
:109280000C40FF88F6FFF6FE0050000800ED00E0FD
:1092900070B5026801239B07114C124D984203D010
:1092A000A04201D0A84203D17026B2434E68324397
:1092B000984203D0A04201D0A84204D103231B024C
:1092C0009A43CB681A4380239A430B691A4302607E
:1092D0008A68C262096881620121416170BD000033
:1092E000000801400014014010B5CB06DB0E01213F
:1092F000046A99408C430462016A9A4011430162F6
:1093000010BD30B58468FF252D021B021343AC430A
:109310000B432343836030BD826870239A430A4322
:1093200007210A438260704730B5026A5208520032
:109330000262026A456883697024A3439C080B6833
:10934000A40023430224A2438C6845601443836134
:1093500049684163046230BD30B5026A10239A4304
:109360000262036A4568826973242402A2430C687E
:1093700024021443202293438A68456012011A4351
:10938000846149688163026230BD30B5026AFF239F
:1093900001339A430262026A4568C3697024A34399
:1093A0009C080B68A400234301246402A2438C6838
:1093B000456024021443C3614968C163046230BD3F
:1093C00030B5026A01231B039A430262036A4568AF
:1093D000C26973242402A2430C68240214430122AC
:1093E000520393438A68456012031A43C461496873
:1093F0000164026230BD30B5036A046A6408640027
:1094000004628469F025AC43120122430A24A34379
:109410000B438261036230BD30B5036A1024A3435D
:1094200003628469036A0F252D031203AC432243B0
:10943000A024A343090119438261016230BD0000E9
:1094400070B501F05BF80D4C0D4D606402E001F069
:1094500055F86064A842FAD10020E0822078002804
:1094600009D0012802D0022805D102E0FCF784FCD3
:1094700001E0FFF75FF900F033FF70BD4800002006
:109480003001CADE10B5818CC90707D001684A686F
:1094900001235B049A43836A1A434A60818C8907DB
:1094A00007D501684A6801231B049A43C36A1A431B
:1094B0004A60818C490707D501684A6801239B04EB
:1094C0009A43036B1A434A60818C090707D50168E8
:1094D0004A680123DB039A43436B1A434A60818C39
:1094E000C90607D50268916801231B039943836B62
:1094F00019439160818C890607D501688A68012328
:109500005B039A43C36B1A438A60818C490612D568
:1095100003685A6801210905046C8A4322435A6092
:10952000026C8A4207D10268516803235B059943A4
:10953000436C19435160818C090607D501684A685C
:109540000123DB04806C9A4302434A6010BD000093
:10955000F8B500260446C667FDF7FEF90546206803
:109560000068124F000709D501212B46002249054A
:109570002046009700F054FA00280DD120680068BA
:1095800040070BD501212B46002289052046009774
:1095900000F046FA002801D00320F8BD20206067C3
:1095A000A067603426740020F8BD0000FFFFFF01B3
:1095B000F8B5184CC826E078002829D16079002831
:1095C00026D101206071144D686B002700281ED041
:1095D000686BC821081A15E01048E168405C6169B1
:1095E00088470F480A21008848430E490880E068F0
:1095F000401CE060E068C82800DBE760696BC820B9
:10960000401A761EE168814201D0002EE4DC6771C9
:10961000F8BD00003000002000000240640C002073
:10962000CE000020DE00002070B5224CE07800283B
:109630003FD1207900283CD1012020711E4EF169D4
:1096400000250906002933DA2156625791420AD1D2
:10965000F06940062CD5A079002829D0A571208971
:10966000401C208124E0A179002903D1A0710A20A7
:1096700000F0D3FC00202056CC2148430F4942186B
:10968000206912181279B262401C00222061A25691
:10969000CC235A43895881420ADC25612078401C3A
:1096A000207020780E2800D12570A078401CA07072
:1096B000257170BD30000020003801403C010020C1
:1096C00010B5806A0022014640314A834A82FEF783
:1096D0006AF910BD70B5846A606FA56F21688968EA
:1096E00000260906002906DA212804D15220065353
:1096F000204600F047F820688068400606D5222DF5
:1097000004D15A200653204600F02CF8E06F1021B7
:109710000843E0672046FEF746F970BD10B50146E4
:109720000968806A0968890614D400225A210A52FD
:1097300001680A68FF2301339A430A6001688A6856
:10974000520852008A6001688A6840239A438A60FE
:1097500020218167FEF7C2FA10BD10B5806AFEF7BE
:10976000BEFA10BD01680A68FF2321339A430A60DC
:1097700001688A68520852008A60202181670021AE
:109780000166704701680A68C0239A430A60202175
:109790004167704770B5164CE278002A0CD12279E7
:1097A000002A09D10122E2700025C82903DC022227
:1097B000A256002A01DCE57070BD0123E356CC22DD
:1097C00053430C4AD1500123E356CC2673439B18D4
:1097D0000A460146181DFBF7D1FC6078401C6070FA
:1097E00060780E2800D16570A078401EA070E2E776
:1097F000300000203C010020F8B504462669A2682C
:10980000E76932436669102000253E4323683243EE
:1098100078491E68784F3E4016431E6023685A6898
:1098200003263603B243E66832435A602368A269CE
:109830008B4201D0266A32439E680B273F02BE430B
:1098400016439E606D4E23686D4AB3420CD1D268B8
:109850009207920F06D0012A38D0022A34D0032A68
:1098600020D11EE001201DE0664EB3420AD1D2682D
:109870000C26324026D0042A28D0082A24D00C2ACC
:1098800010D10EE08B420DD1D66803229202164011
:1098900018D001229202B61A18D0B61A14D09642E5
:1098A00000D10820564A0126403A574FF6038B4212
:1098B00036D100280CD002280DD0042812D0082858
:1098C0001FD11CE00020EDE70220EBE70420E9E7D0
:1098D000FDF7FAFB08E01068C00601D5384605E040
:1098E0004A4803E0FDF710FC002873D0626851007D
:1098F0005118814205D81103814202D303E030465A
:10990000F4E7012566E0010E060250080023301836
:109910005941FBF703FC03210902411A3C4A55E077
:10992000E169B14232D1030000F081F909070A0D63
:1099300006250606062B0600E3E7FDF7C5FB1CE03F
:10994000FDF7D2FB19E010686168C00602D548082F
:10995000304A01E0304A48088018FBF7C9FB80B262
:1099600001462E4A10399142CBD8511C01400007C4
:10997000400F08432CE0FDF7C7FB616840004A0830
:10998000EAE76168012248081204E5E7030000F0F5
:109990004EF909070A0D06260606062C0600B0E752
:1099A000FDF792FB1DE0FDF79FFB1AE01068616870
:1099B000C00602D54808C01902E014484A08101829
:1099C000FBF796FB80B20146144A1039914298D8B1
:1099D0002168C8600020206660662846F8BDFDF753
:1099E00093FB61684A088018EAE7616848088019B3
:1099F000E6E7000000480040F369FFEF003801404F
:109A0000401002400044004000093D000024F400E2
:109A1000FFFC0F0000127A000048E801EFFF000091
:109A2000FFB581B017460E4604460A9D09E0681C42
:109A300007D0FCF791FF0499401AA8420CD8002DDA
:109A40000AD02068C1693046884318D00020B84247
:109A5000EDD0002005B0F0BD20680168FF22A132E2
:109A60009143016020688168490849008160202095
:109A70006067A0670020603420740320EAE70120BB
:109A8000E5E7000010B504491020096808620248A3
:109A9000FDF78AFF10BD00007415002001490D205C
:109AA000887070473000002010B507480A22418AAC
:109AB00051434184FEF7BCFCFEF7D4FDC8220349A4
:109AC0000348FEF7AFF810BDBC000020640C002076
:109AD00074150020F8B53D4C002321783C4A1D4602
:109AE000082910D0072945D006294ED0052950D085
:109AF000042951D0032952D0002954D0012956D02D
:109B0000022958D059E0A17800264A1F04E0304FBE
:109B1000BF5DFB189BB2761C9642F8DB667927790D
:109B20009A195118E3786278C9188918C919401828
:109B3000C0071AD0012E14D0022E16D12548244970
:109B4000C018FBF71BFB00F0BBFF642000F05EFABF
:109B5000BFF34F8F21492048C860BFF34F8F00BF2C
:109B6000FDE759081046FFF79DFA2570E570A570CE
:109B7000A571F8BDA1795054491CC8B2A071A17853
:109B8000491F8842F5D1082001E06070072020704D
:109B9000F8BDE0700620FAE760710520F7E7A070D5
:109BA000E5700420F3E7552807D10120EFE7AA2844
:109BB00003D10220EBE7032803D02570E570A570E0
:109BC000F8BD032020702071F8BD0000B300002014
:109BD0008C1300202C0D00200400FA0500ED00E09D
:109BE0000FB410B503A9044B044A029800F002F91F
:109BF00010BC08BC04B018473DA80008FC000020B9
:109C00002021020C01D010211046020A01D010467A
:109C10000839020901D01046091F820801D01046F8
:109C2000891E420801D0881E7047081A704730B458
:109C30007446641E2578641CAB4200D21D46635DE9
:109C40005B00E31830BC184702E008C8121F08C1C7
:109C5000002AFAD170477047002001E001C1121FAD
:109C6000002AFBD1704708B50021684601706B4699
:109C7000012202212C2000F081FD022168460170A2
:109C80006B4601222C2000F079FD08BD38B5044652
:109C90006D20694608706B46012207492E2000F0AE
:109CA0006DFD0649002C01D0054A00E0054A2E2032
:109CB00000F04AFD38BD000006080000061800004C
:109CC000070600000716000038B504466B4602225E
:109CD0000021362000F018FCB3212300FFF7A7FF76
:109CE0000E0F08153A3A3A3A1C273A3A2F34483AB6
:109CF00000216846017040784108490014E0694637
:109D0000087880088000401C04E0694608788008D4
:109D10008000801C08701DE0684602780A404832C6
:109D200002704178802001436846417012E0684625
:109D300002780A40027040784106490EF4E769460D
:109D400048780221084303E069464878FD2108402D
:109D5000694648706B4601220021362000F00EFD56
:109D6000012200AB11463620013300F007FD38BD5B
:109D700069460878CF21084069462030CAE708B50F
:109D8000032168464170012101706B4602220021C7
:109D9000362000F0F3FC0122D20306212D2000F032
:109DA000D3FC012000F032F90120FFF78DFF08BD40
:109DB00008B5020A69464A7008706B4602220421FF
:109DC0002D2000F0DBFC0320694608706B46012261
:109DD00006212D2000F0D2FC0020694608706B4659
:109DE000012206212D2000F0C9FC0A212D2000F0BF
:109DF00071FB08BDFFB58DB00446002506E025289F
:109E00000AD0109A0F999047641C6D1C2078002886
:109E1000F5D1284611B0F0BD00270121484A00972E
:109E200000E00743641C23780846203B984010421A
:109E3000F7D120782E2817D1042007436078641CBE
:109E40002A280CD10E98641C02C800910E900BE0D9
:109E500000990A22514330394018641C0090207840
:109E6000014630390929F3D920780028D1D0642857
:109E700008D0692806D075281ED0109A0F999047EF
:109E80006D1C5BE00A200E99019001C90E9100281B
:109E900002DA40422D2102E0390504D52B216A4621
:109EA0001172012103E0F90704D02021F7E70BAE7E
:109EB0000B910DE00021FAE70A200E99019001C9EB
:109EC0000E91F7E70199FBF713F93031761E3170E7
:109ED0000028F7D103A8801B20300190780701D516
:109EE000009801E0012000900199884201DD401AAC
:109EF00000E000200027009006E002A8109AC05D54
:109F00000F9990476D1C7F1C0B988742F5DB04E08E
:109F1000109A30200F9990476D1C0099481E0090B0
:109F20000029F5DC05E03078109A761C0F999047EF
:109F30006D1C0199481E01900029F4DC641C65E742
:109F400009280100F8B54A002B4B520DD6182B4AB0
:109F50000C460546142E2BDA002E12DA284BFBF79E
:109F6000D5F900221346FBF7FBFC40D2002C03DAA4
:109F70000124E40700253AE02046284337D0214C4D
:109F800014E0214F0B46F7403B402B4331D01C4B94
:109F9000FBF7BCF900221346FBF7E2FC27D2002CAA
:109FA00003DD01200005F0400419BC4300251EE03C
:109FB000332E1EDC33460027143BFF43DF4038427C
:109FC00017D00F4BFBF74CFA00221346FBF7C8FCE7
:109FD0000DD2002C0ADD142E0CD03420811B012060
:109FE00088404019A84200D2641C0546BD43214662
:109FF0002846F8BD641CF9E701FCFFFF9C7500884A
:10A000003CE4377E0000F03FFFFF0F007D2110B5DC
:10A01000C900484300F001F810BD002140E000BF36
:10A0200000BF00BF00BF00BF00BF00BF00BF00BF38
:10A0300000BF00BF00BF00BF00BF00BF00BF00BF28
:10A0400000BF00BF00BF00BF00BF00BF00BF00BF18
:10A0500000BF00BF00BF00BF00BF00BF00BF00BF08
:10A0600000BF00BF00BF00BF00BF00BF00BF00BFF8
:10A0700000BF00BF00BF00BF00BF00BF00BF00BFE8
:10A0800000BF00BF00BF00BF00BF00BF00BF00BFD8
:10A0900000BF00BF00BF00BF00BF00BF00BF491C22
:10A0A0008142BCD370470000FEB5044600200190F9
:10A0B00000906079734940000E5A61782578491EF6
:10A0C0007148CFB20163042D77D0072D75D00021E0
:10A0D0000291217801736C49E37901229205896923
:10A0E000002B6CD0914381616748217A4173217ABA
:10A0F00082698907890B0A4382610021042000F0EC
:10A100002EFB324661492E2000F01EFB3846FFF739
:10A11000BDFD5F4E0522705D810040185D4943180A
:10A1200007212B2000F02AFB5B49029801220B1823
:10A130000B21282000F022FB705D584980000A584E
:10A140000C21282000F00BFBE079554980004018D5
:10A15000A1794900425A0221272000F0F5FA51481E
:10A160007E00825B0421272000F0EEFAE0790028CF
:10A1700029D0A07804282CD02820694608722022F3
:10A180000621272000F0E0FA02AB01222621272039
:10A1900000F0F4FA444938014018E1788900425847
:10A1A0000821272000F0DBFAA17A601C627A0902FC
:10A1B000114313D016E000E001E0012188E71143CC
:10A1C000F608816190E764220621272000F0BCFA9E
:10A1D000E0E71020694608720246D1E73349017270
:10A1E000090A4172417A007A0A020243202127209B
:10A1F00000F0AAFA2E4F0C2123203A6800F0AFFAA3
:10A20000F01982880421232000F09EFAA07900280A
:10A210000BD0E0792749012243180021212000F0CA
:10A22000ADFA03200190012000902A07120F1001BF
:10A230000243607800218007000B0243019800056B
:10A2400002430098400402432079C00640090243BB
:10A250006079C00602431F2000F081FAA07861787F
:10A260000123084302040848DB030261E179490342
:10A2700019430A4302610021082000F070FA00200F
:10A28000FEBD00008CAB0008000100200428000087
:10A2900034AB0008010000201F0000203CAB000888
:10A2A0005CAB000868AB00086CAB00084110000014
:10A2B00054AB00082100002038B50C4607498A8BB2
:10A2C000002102432C2000F03FFA684604706B46E0
:10A2D000012206212C2000F051FA38BD0001002097
:10A2E00010B5FFF7C0FC10BD10B5044604213620A0
:10A2F00000F0F0F80121C902002C01D0084300E071
:10A30000884302460421362000F029FA10BD0000DF
:10A3100038B540206946087000210E2000F0DAF8B8
:10A320000446002211460E2000F019FA6B46012265
:10A3300000210D2000F022FA074A00210F2000F032
:10A340000EFA00F0E7F9224600210E2000F007FA8D
:10A3500002480021017338BDF8FF272420010020A6
:10A360007CB505460420694608704B4C002060759A
:10A3700021462031206348710873A0836063A06385
:10A3800000F0BCF8454E206002E000F0B7F8206015
:10A39000B042FAD10020FFF797FC4148007824280A
:10A3A00001D9243806E00621FAF7A2FE0622101A87
:10A3B00040010843020601040A4301020A43024322
:10A3C00000211E2000F0CBF96B4601220021242041
:10A3D00000F0D4F91E20FFF7EBFC86B2300AA07320
:10A3E0000420FFF7E5FC0006000E0DD002206946B0
:10A3F000087101AB012212212D2000F0BFF9A08BC2
:10A40000012109030843A08300F078F820600620AA
:10A41000FFF7CEFC60600720FFF7CAFCA060F006E3
:10A42000C00E207501D110202075C0B200F0E2F9F5
:10A43000E80707D0FFF7A3FCA08B0121C90208435E
:10A44000A0830AE00521362000F02EF815490840C7
:10A4500002460521362000F077F90120FFF734FC91
:10A460000021042000F036F8A0610021262000F031
:10A4700031F815218903084302460021262000F007
:10A480006EF900222621362000F05EF900F036F841
:10A49000206000207CBD0000000100203001CADEE9
:10A4A00000000020FFFD000038B5094C89B280B2E1
:10A4B0006B46022200F028F8002806D16846407852
:10A4C000010268460078081884B2204638BD0000B2
:10A4D000FFFF000038B50024E44389B280B26B4628
:10A4E000042200F011F8002806D103216846435CDD
:10A4F0002202D418491EFAD5204638BD10B50021D5
:10A500000846FFF7E7FF10BD38B5002909D0402401
:10A5100020436C462070C8B27F2906D860700220A4
:10A520000AE069460870012006E0802420436C465A
:10A530006070C809A0700320694600F09BFA38BD1E
:10A5400010B5144603460A4621461120FFF7DCFFEA
:10A5500010BD10B50346052200211520FFF7D4FFDA
:10A5600010BD10B501210620FFF7B4FF10BD10B5D6
:10A570000346052200211720FFF7C6FF10BD38B59E
:10A58000054600206946087000F0C4F8FF24013435
:10A590002246002D01D00322120200210D2000F0DE
:10A5A000D3F8002D13D06B46012203210F20FFF7B3
:10A5B000ABFF68460078000709D5FFF7A9FE2246E1
:10A5C00000210D2000F0C0F80020C04338BD00205D
:10A5D00038BD10B5024601210A2000F0C0F810BDB8
:10A5E00010B5044600211A20FFF774FF000D220366
:10A5F0000005120B024300211A2000F0B0F810BD34
:10A6000010B5024602492E2000F09EF810BD000051
:10A6100004180000F8B505466B460122032104200A
:10A62000FFF772FF0126114C3607002D0DD02A4688
:10A6300000210C2000F088F86946087810210843B2
:10A6400069460870A069304307E069460878EF2141
:10A65000084069460870A069B0430B46A06101221A
:10A660000321042000F08AF8F8BD0000000100205A
:10A6700010B502460021182000F066F810BD000059
:10A68000F8B50746002568460570B807204C2E46E9
:10A6900000280ADA8020694608706B4601220021F2
:10A6A0000D2000F06BF801202073F8076946087848
:10A6B00021D006210843694608706B46012200211B
:10A6C0000D2000F05BF803210F20FFF7EDFE812144
:10A6D000C900084219D04020694608706B46012223
:10A6E00000210D2000F04AF80020FFF7FDFD0025B5
:10A6F0002673ED4309E002210843694608706B4662
:10A70000012200210D2000F039F82846F8BD000094
:10A71000200100201CB56B46012203210F20FFF70A
:10A72000F3FE684600784022C1091040C90140008C
:10A73000814208D0012069460871024601AB03211D
:10A740000D2000F01BF81CBD08B56B461A70120AEC
:10A750005A7089B280B2022200F010F808BD38B5F4
:10A7600000236C46E254120A5B1C042BFADB89B20C
:10A7700080B22346042200F001F838BD38B58024A9
:10A78000002909D0C02528436D462870C8B27F290A
:10A7900007D86870022009E020436946087001204C
:10A7A00004E020436870C809A8700320694600F0DF
:10A7B0009DF938BD10B51446012312189B029A4228
:10A7C00002D90020C04310BD0B46821E214609203D
:10A7D000FFF7D4FF002010BD10B5054A89051269A6
:10A7E00001430A4300210820FFF7B9FF002010BDF4
:10A7F0000001002038B504466B4601220E212B20B3
:10A80000FFF782FE68460078E10640094001C90E64
:10A810000143684601706B4601220E212B20FFF791
:10A82000ADFF38BD10B5002142541C06120A224368
:10A830001B0A491C0429F7DB10BD000013B50123D6
:10A840001A4669460248FDF74BFA00981CBD000005
:10A8500074150020FCF78EF8FEF7A4FCFDF7FCFD54
:10A8600041494248002522C005608561C5614049D3
:10A870000562C1600838FCF7B3F9FDF7D9FDFDF7B3
:10A88000F1FEFDF78DFEFDF79FFD0526012236073F
:10A89000D1033046FCF759F8FEF716FBFDF798FC9C
:10A8A000FBF71EF9FBF7F6F8FDF78AFA0721B0155A
:10A8B000FFF702FDFFF714FD2E4C0A21608A0122EA
:10A8C0004843608411033046FCF73FF82748C8220C
:10A8D0002949C430FDF7A6F9284F294EE078002811
:10A8E0003ED0E07900283BD0FEF75CFCE570FBF73A
:10A8F0000FFB20700F280AD9012211033046FCF704
:10A9000024F8FEF79DFD00220121090309E0012240
:10A9100051033046FCF719F8FEF792FD00220121A1
:10A9200049033046FCF711F8FDF784FB608C0028E2
:10A9300001D0401E60841348618C00780843CDD15B
:10A940003878002801D00328C8D140213046FBF7D1
:10A95000F7FF0028C2D101210846FCF733FABDE712
:10A96000FDF768FBBAE70000007C0040B01400204F
:10A97000FFFF0000BC000020640C00205A000020F3
:10A98000000400503600002010B586B01748FCF7D0
:10A99000ACF814216846FAF70AFC15480090032029
:10A9A000019000200290052069460007FBF70CFF8C
:10A9B00069461048FBF708FF69460F48FBF704FF9C
:10A9C00001210846FCF7FEF9FF2401342046FCF77C
:10A9D000D1F90A4908680422104308602046FCF7B0
:10A9E000D9F9FCF7DFF906B010BD0000B014002063
:10A9F000FFFF0000000400500008005000700040FD
:10AA000010B50122920218491848FBF7DFF81648E2
:10AA1000174902888A4226D0018004218180FF21C3
:10AA2000F531C1800A21018100211E224181D243DA
:10AA300082810122C2810184018241828182C1829C
:10AA4000018381834323C3860223038778234387BB
:10AA50008287C2870246403291801184518491845A
:10AA6000C18300F02DF810BD2C0D002000FC000863
:10AA7000AA550000F0B58C460025102605210907CF
:10AA80008E620E4C08E067467F5DE760A768FF07AF
:10AA9000FCD0E7681F706D1C8542F4DB0020074680
:10AAA00006E0E760A568ED07FCD0E5681D54401C92
:10AAB0009042F6D38E610020F0BD000000300140CE
:10AAC00070B572B60124074DA40221462846FBF753
:10AAD00063F8002804D0224603492846FBF700F912
:10AAE00062B670BD00FC00082C0D0020F0B50025FA
:10AAF000102605279C463F070B46BE620C4C06E01D
:10AB0000595DE160A168C907FCD0E1686D1C854210
:10AB1000F6DB002007E06146095CE160A168C90737
:10AB2000FCD0E168401C9042F5D3BE610020F0BD2E
:10AB3000003001400000010203040005405C0000F9
:10AB4000A05C0400C06C0800805C0400E03F1E00B4
:10AB5000E07D1E0007A9022570889B880A00160068
:10AB6000010006000100020087008D002D001A314F
:10AB700052001A339A001A351D011A376B003B3107
:10AB8000BE003B335E013B3596023B3700009959CE
:10AB90009959EB518F421E45142E0080EB51F52838
:10ABA0003333E13A703DE13AC235852BC235333358
:10ABB000C235C235AE47E13A5138A33051380000B2
:10ABC0000000000000000102030406070809030456
:10ABD00006080C10182030000000000102030400D9
:10ABE00000AC00080000002000010000489C0008A4
:10ABF00000AD000800010020A0190000589C0008CA
:10AC000000070400091E08054008260910400856E0
:10AC100008054008261D040008BE1D040008BED813
:10AC2000BC401008010000000000C8420000000005
:10AC30000000000000000000000000000000000014
:10AC40000000000000000000010000000000000003
:10AC50000000000000000000000000008C0A00005E
:10AC600000000000000000000000000000000000E4
:10AC700000000000000000000000000000000000D4
:10AC800000000000000000000000000000000000C4
:10AC900000000000000000000000000000000000B4
:10ACA0000000000000000000020214000909010277
:10ACB0000081000000000000010000000000000012
:10ACC0000000000000000000000000000000000084
:10ACD0000000000000000000000000000000000074
:10ACE0000000000000000000000000000000000064
:10ACF0000000000000000000000020000000000034
:04000005080050C1DE
:00000001FF
